:100000008A150028FF3FFF3F03138312F8010830D1
:10001000FC00700DF80D7408F80203181128F80799
:100020000310F00DFC0B0928080000000000080078
:10003000040803138316CF0083122008840084135E
:1000400000088316CE00CE134E134E0880004F08D2
:1000500084000800031383127008F100F0010830D7
:10006000FC007108F40C03183928FC0B3228F1014C
:10007000003403103E28F40C0318F107F10CF00CC7
:10008000FC0B3B28080003138316CF014E08093CE4
:1000900003186A280A30F4004E08F00004207008A3
:1000A0008316CF007008D000D00D5010D00D501026
:1000B000D00D5010D00D50105008CF000A30F40071
:1000C0004E08F00004207808F000700883165004F1
:1000D000CF006C284E08CF004F08F0000800031333
:1000E00083164E08CF004F088400CF0A0008F000A6
:1000F0007008031D73284E084F02F0000130F00213
:10010000F101031CF1030800003003138316981853
:100110000130F1007108003A031D90280000842886
:100120004E088312990008000313831295011712D9
:10013000971208000313831222088A002308820002
:10014000080003138312FB01FA01F9018030F80063
:10015000FD01F11FB128F109F009F00A0319F10AB4
:10016000FD0AF51FB928F509F409F40A0319F50A7F
:10017000FD0AF10CF00C031CC6287408F907750879
:100180000318750FFA070318FB0A0310F01FCE2897
:100190007408FA070318FB0A7508FB07FB0CFA0C36
:1001A000F90CF80C031CB9287D1CE128FB09FA099D
:1001B000F909F809F80A0319F90A0319FA0A0319DF
:1001C000FB0A7B08F3007A08F2007908F10078084E
:1001D000F00000000800031383122008840083133A
:1001E00080171520001715201820801315201820BF
:1001F00000130800083003138316CB00CC018312D0
:1002000020088400831383164B0803192129152025
:1002100015201820001315204A0803190F2918204B
:10022000CA0D031C162984178017182984178013F8
:100230000000152000178413001F1C298417CB030E
:100240000329CC0115201820000000131520801769
:10025000152015204C0803192D2900178413001FA1
:100260002F29CC0115208413801B4C141520152038
:10027000152015201520152015201520182084176D
:10028000001380134C08F0000800031383122008A9
:100290008400831318208013152000178413001F77
:1002A0004F2984171520152015201520801715209B
:1002B0000800083003138316CB00CC0183122008FA
:1002C0008400831383164B08003C03187D291520F6
:1002D0000000801715204C0803196E29001784139D
:1002E000001F7029801B0314801F0310CC0D1520E4
:1002F000182084170013CB036229801715204A08A1
:100300000319832918204A0803198729801300003C
:10031000152000178413001F8B298417152018201F
:1003200000131520182080134C08F00008000F302F
:10033000031383164A05CB004A08F000F00CF013B3
:10034000F00CF013F00CF013F00CF0130A30F40082
:100350002A2083164B08F0070800031383164A0867
:10036000CE00432070088312A400F0307005A50071
:10037000A6010030A6050030A6000430F2002508D2
:10038000F0002608F10072080319CD29F10CF00CD9
:10039000F113711BF117FF3FC4297008A500710804
:1003A000A6003030F0070318F10A7008A5007108A4
:1003B000A60027088400700880000F302405A500DF
:1003C000A6010030A6050030A60030302507F20057
:1003D00026080318013FF3000030F3077208A50058
:1003E0007308A600270AF0007008840072088000D5
:1003F00002302707F00070088400280880000330CE
:100400002707F0007008840080010800031383169A
:100410004A08CC004C0884000008F000700803195A
:10042000132ACC0A0A2A4C08F100CC0A4B08840093
:10043000CB0A0008F0007108840070088000710881
:1004400084000008F0007008031D132A4A08F00019
:1004500008000313831229088316CE006F2070084A
:10046000CB00CA014A0883122907840000088316BA
:10047000CE0084208316CA0A80304A06F0008030FD
:100480004B067002031C322A08000E30031383123D
:10049000FA00FA0B492A0000080003138312F8013E
:1004A000F9011030FC00710DF80DF90D7408F80217
:1004B0007508031C750FF9020318652A7408F807FC
:1004C00075080318750FF9070310F00DF10DFC0BFB
:1004D000532A080003138312710DF80DF90D7408E7
:1004E000F8027508031C750FF902F00DF10D0F30BD
:1004F000FC00710DF80DF90D7408701C852AF802C6
:100500007508031C750FF9028A2AF8077508031885
:10051000750FF907F00DF10DFC0B792A7018962A6A
:100520007408F80775080318750FF907000008002C
:100530000313831286018316860185309F00FF30E6
:10054000831285001F30831685008312870183166E
:1005500087018312121463308316920094200800DE
:1005600003138316031383164608F200C60A4708CE
:10057000F0004808F100C70A0319C80A700883127E
:10058000A3007108A2000A08A1009A20F000210827
:100590008A007208840070088000720884000008D5
:1005A000F00070080319D52AB02A08004D346934C8
:1005B0006B3472346F344334203438343734363447
:1005C0002034503457344D345F34543465347334EC
:1005D00074345F34303438342E346334203430345F
:1005E000373431343034323438340A340D34203432
:1005F000003408005034613475346C3466346A3425
:1006000075346A346F340A340D340034080003132F
:1006100083160711831212150C3097040800031378
:1006200083126E088316C600031383164608F10072
:10063000C60A83126F088400EF0A0008F0007108F0
:10064000840070088000710884000008F0007008C1
:10065000031D142B6E08F000080003138316120804
:10066000013FF000F1010318F10A83126E08F40053
:10067000F501A1200630F2007008F4007108F500C1
:1006800072080319482BF50CF40CF513FF3F412BAE
:100690007408F000F00D7010F00D7010F00D701077
:1006A000F00D701030307005F3007408F00075081C
:1006B000F100F10CF00CF113F10CF00CF1137008D7
:1006C00095000F3097057308970408004D344134A6
:1006D0004A343A342034413441344D344D34443476
:1006E00044344A344A34483448344D344D340A345E
:1006F0000D3400340800EB20D030CA00FA208312F9
:100700006E088316CA00FA2083126F088316CA0087
:10071000FA204521EB20C60180304606F0008030EB
:10072000033A70020318AD2B0330FB00FF30FA00D0
:10073000FB0B9B2B9E2BFA0B9B2B982B9630FA00D6
:10074000FA0BA02B0000CA01FA2070080319AA2B8B
:10075000EB20AB2BAD2BC60A8C2B452108000030BB
:10076000031383128C1A0130F1007108F0000800A5
:10077000031383121A08EE00981CC02B18121816C7
:100780006E08F0000800031383122908840080011A
:1007900045218230FB00FF30FA00FB0BD02BD32B1E
:1007A000FA0BD02BCD2B8730FA00FA0BD52B00009B
:1007B0000000EB20D030CA00FA20CA01FA20EB205A
:1007C000D130CA00FA200130CA00592170088312C2
:1007D000A500A60125088316CA0097217008831278
:1007E000B00001308316CA00592170088312A50099
:1007F000A60125088316CA00972170088312AF004E
:1008000001308316CA00592170088312A500A60181
:1008100025088316CA00972170088312AE000130A4
:100820008316CA00592170088312A500A601013061
:100830008316CA00592170088312A500A601250855
:100840008316CA00972170088312AC00013083160A
:10085000CA00592170088312A500A6012508831635
:10086000CA00972170088312AB008316CA01592170
:1008700070088312A500A60125088316CA009721D7
:1008800070088312AA0029088400800129088400C6
:1008900080014830A8002E088316CA00AD2129081F
:1008A0008316CA00831227088316CB0006224D3018
:1008B0008312A8002F088316CA00AD2129088316C9
:1008C000CA00831227088316CB00062253308312F6
:1008D000A80030088316CA00AD2129088316CA0073
:1008E000831227088316CB00062229220930CE0066
:1008F00084200800031383129F01C0309F048316D5
:100900001F179F1783126E08F000F00D7010F00D86
:100910007010F00D701070089F041F1445221F15F1
:100920001F1D942C0000902C1F100830F2001E0890
:10093000F000F10172080319A22CF00DF10D7010F6
:10094000FF3F9B2C83161E08F0040030F1040800C2
:100950000313831648088400203080002030840A66
:100960008000840A8000840A8000840A80000130AC
:100970008312EE0083164708003C031DC12C460875
:10098000093C0318C52C8312EE0A83164708003C65
:10099000031DCC2C4608633C0318D02C8312EE0AAE
:1009A00083164708033C031DD72C4608E73C031871
:1009B000DB2C8312EE0A83164708273C031DE22C2A
:1009C00046080F3C0318E62C8312EE0A0530831606
:1009D0004807F000700884008001840383126E08C9
:1009E000003C03181A2D0A30F400F501831646085E
:1009F000F0004708F1004D227808F0007908F10076
:100A000070088000000883164602F0000030031CC6
:100A1000013F4702F1000A30F400F5014D22700851
:100A20008316C6007108C700303080078403831224
:100A3000EE03EE2C0800F030031383126E05F20073
:100A40007208F000F00CF013F00CF013F00CF0133F
:100A5000F00CF01330307007F10071088316C600F7
:100A60007108393C0318362D0730C6070F30831242
:100A70006E05F00030307007F10071088316C70072
:100A80007108393C0318462D0730C7074608CE00C9
:100A9000842083164708CE00842008002E300313DC
:100AA0008312B1002E30B2002E30B3002E30B400CD
:100AB0002E30B5002E30B6002E30B7002E30B800E4
:100AC0002E30B9002E30BA002E30BB002E30BC00C4
:100AD0002E30BD002E30BE002E30BF002E30C000A4
:100AE0002E30C1002E30C2002E30C3002E30C40084
:100AF0002E30C5002E30C6002E30C7002E30C80064
:100B00002E30C9002E30CA002E30CB00CC0131303F
:100B1000A9002E30CD002E30CE002E30CF002E304A
:100B2000D0002E30D1002E30D2002E30D3002E3007
:100B3000D4002E30D5002E30D6002E30D7002E30E7
:100B4000D8002E30D9002E30DA002E30DB002E30C7
:100B5000DC002E30DD002E30DE002E30DF002E30A7
:100B6000E0002E30E1002E30E2002E30E3002E3087
:100B7000E4002E30E5002E30E6002E30E7002E3067
:100B8000E800E9014D30A7002F308316A0002F3078
:100B9000A1002F30A2004430A3004830A4004D3003
:100BA000A5005330A600A70108000313831698166A
:100BB00090308312980083168717071383128C1EB8
:100BC000E42D1A08EE00DE2D0800031383126E08D0
:100BD00084000008EF00EF136F136F088000841784
:100BE0000408A000801700178413001FF52D0800CB
:100BF00003138312FB01FA01F9018030F800F10CB4
:100C0000F00C031C0C2E7408F90775080318750FF7
:100C1000FA070318FB0A0310F01F142E7408FA07D2
:100C200075080318750FFB07FB0CFA0CF90CF80C90
:100C3000031CFF2D7B08F3007A08F2007908F1000D
:100C40007808F000080003138312FD01F901F80190
:100C5000710870040319003471087506FA00FA1B54
:100C6000FD09FB01F51F392EF409F509F40A0319F2
:100C7000F50AF11F402EF009F109F00A0319F10AF3
:100C800071087504FA00FA1B552E6A227B18682E2B
:100C9000FD1F0034F009F109F00A0319F10AF809FF
:100CA000F909F80A0319F90A0034F51F642EF11B3B
:100CB000602E7108F9007008F800F101F001482E6B
:100CC000F101F001F00A0034F109F009FB0A452EA8
:100CD000F80A0319F90A74087802031D482E7508EA
:100CE0007902031D482EF901F801F00A0319F10AEF
:100CF000F11F482E0000FF340800FF3FFF3FFF3F79
:100D0000FF3FFF3FFF3FFF3FFF3FFF3FFF3FFF3FF3
:100D1000FF3FFF3FFF3FFF3FFF3FFF3FFF3FFF3FE3
:100D2000FF3FFF3FFF3FFF3FFF3FFF3FFF3FFF3FD3
:100D3000FF3FFF3FFF3FFF3FFF3FFF3FFF3FFF3FC3
:101000008A114E258A154D30A8006F30A9006E3028
:10101000AA007430AB006530AC006530AD00203004
:10102000AE000A30AF000D30B000B1014330B20065
:101030006F30B3006E30B4007330B5002030B600AE
:101040003D30B7002030B800B9012030BA004D3033
:10105000BB006530BC007330BD002030BE00653081
:10106000BF006E30C0002030C1002530C2003D30CE
:10107000C3002030C400C5018A1198228A1533307C
:101080008316990018158A11D5258A152908831603
:10109000C600D630C7000230C8008A11B0228A15B7
:1010A0008A1129228A15831229088316C600FA306C
:1010B000C7000230C8008A11B0228A158A1129227D
:1010C0008A15831285128A1107238A152908EE00D2
:1010D000A830EF008A110F238A157008A9008A1121
:1010E00029228A1506308312EE008A11E5258A1519
:1010F000EA01FF306A02031896286A08EB006A08C2
:10110000EE008A112D238A158230FB00FF30FA0091
:10111000FB0B8B288E28FA0B8B2888288730FA0047
:10112000FA0B902800000000EA0A792885160030A2
:1011300005190130F2007208003A031D012929083F
:101140008316C6006630C7000330C8008A11B0227B
:101150008A158A1129228A158312EE01EF018A115C
:101160007B238A1506308312EA006A08003C0318C4
:1011700001298A11AF238A1570080319B9288A1129
:10118000B8238A157008EC0070088316CE008A1107
:1011900084208A1530306C02F2007208EB0072086D
:1011A000A400A40D2410A40D2410A40D2410A40D3B
:1011B00024108A11AF238A1570080319D9288A11BF
:1011C000B8238A157008EC0070088316CE008A11C7
:1011D00084208A1530306C02F0007008EB00F0308B
:1011E000A4057008A4076C081B3A031901296A08B2
:1011F000EE002408EF008A117B238A158312EA038C
:10120000B5280D308316CE008A1184208A158512E8
:101210008A11C3238A15EE018A117A248A1570086F
:101220008312A5007108A6007008F2007108F3008F
:10123000F30CF20CF313731BF317F30CF20CF31310
:10124000731BF3177208EB002908EE00B230EF00B1
:101250008A110F238A157008A9008A1129228A157C
:10126000831225088316C600831226088316C7003A
:10127000831229088316C8008A11A8248A158A11A6
:1012800029228A1583126B08EE008A112D238A15F4
:101290002908EE00BA30EF008A110F238A15700872
:1012A000A9000130EE008A117A248A150A30F40070
:1012B0000030F5008A11F8258A157008A50071081C
:1012C000A6006630F4000030F5008A1123268A1546
:1012D0007008643CED008A1129228A1583126D087A
:1012E0008316C600C701831229088316C8008A1115
:1012F000A8248A158A1129228A150930CE008A115C
:1013000084208A156D08EE008A111B258A150D3080
:101310008316CE008A1184208A1585160330FC00BE
:10132000FF30FB00FF30FA00FC0B97299E29FB0BD6
:101330009A299D29FA0B9A29972994298C30FB0028
:10134000FF30FA00FB0BA529A829FA0BA529A22931
:10135000A130FA00FA0BAA29000000000729AF29E2
:02400E007A3FF7
:00000001FF
